:100000003EC1000058C1000056C1000054C10000AC
:1000100052C1000050C100004EC100004CC10000A0
:100020004AC1000048C1000046C100000C946A0BA0
:1000300042C1000040C100003EC100003CC10000C0
:100040003AC1000038C1000036C1000034C10000D0
:1000500032C1000030C100002EC100002CC10000E0
:100060002AC1000028C1000026C1000024C10000F0
:1000700022C10000F002F50200030A031003160378
:100080004403500355035A0369036E037903950330
:10009000A803AE03B603BA03BC03C6034604660452
:1000A0007C048B0471056D057505790573056F0575
:1000B00077057B05370C5A0C450D5A0C450DA10CE4
:1000C000C30C450D160D280D2203690062006D005A
:1000D0002D00630061007000730065006E00730006
:1000E00065002D00750073006200000022035400BB
:1000F0006F006D00200057006F006E0067002D003C
:1001000043006F0072006E0061006C006C00000024
:100110000403090409025400030100A03209040089
:10012000000103010100092111010001222500073E
:1001300005810308000A0904010001030000000909
:1001400021110100012220000705830308000A098C
:10015000040200010300000009211101000122BE78
:10016000000705820319000A120110010000002097
:10017000810402000100010200010600FF0901A143
:10018000010902150025FF7508950881020903156C
:100190000025FF750895089102C005010906A10117
:1001A0000508190129031500250195037501910220
:1001B000950175059101050719E029E7150025014D
:1001C00095087501810205071900293115002501DF
:1001D0009532750181029501750181010507193379
:1001E000299B15002501956975018102950175010D
:1001F00081010507199D29A41500250195087501A0
:1002000081020501198129831500250195037501D6
:100210008102050C19B029B8150025019509750151
:100220008102050C09CD09E209E909EA0A8A010AF5
:1002300092010A94010A21020A23020A24020A25D1
:10024000020A27020A2A0215002501950D7501816F
:1002500002950175028101C005010906A101750120
:100260009508810195017508810195057501910138
:10027000950175039101950675088101C00011244F
:100280001FBECFEFD4E0DEBFCDBF11E0A0E0B1E0F4
:10029000E6EEFFE102C005900D92A635B107D9F751
:1002A00014E0A6E5B1E001C01D92A133B107E1F76A
:1002B0008FD00C94F10FA4CE49C33FC380E291E0EC
:1002C0000E94AE0E80E191E00E94AE0E80E091E0CF
:1002D0000E94AE0EE2EEF0E080818460808308959B
:1002E00080E291E00E94780D80E191E00E94780D1B
:1002F00080E091E00C94780D80912E0190912F0177
:10030000009729F0019790932F0180932E018091FF
:100310001E0190911F01009729F0019790931F01F2
:1003200080931E0180910E0190910F01009729F09A
:10033000019790930F0180930E010FC30F931F93AA
:10034000CF93DF93FC01C901E80121E0E032F2071D
:1003500011F478D305C021E0E031F20721F4CED1C9
:1003600088E090E005C066817781DDD389E190E087
:100370009983888380E0DF91CF911F910F91089539
:10038000AC01C90121E04032520709F482C4405156
:10039000514009F418C180C484B7877F84BF88E1C5
:1003A0000FB6F89480936000109260000FBE90E04A
:1003B00080E80FB6F89480936100909361000FBEBF
:1003C0003AD00AD7B5D20DD75E9A5E980C945B0BE3
:1003D000E3DF789428D308D67CD60DD38FE19EE452
:1003E0000197F1F700C0000049D0809185019091FC
:1003F0008601019609F408D552D4809128048823F7
:1004000021F080912804853039F4809126048823D6
:1004100019F0C1D58111FBD680E291E00E94C10E96
:1004200080E191E00E94C10E80E091E00E94C10E47
:100430000E945E0DE1CFC1D6289A0895CF93DF9335
:1004400090938601809385012898EC01CC0FDD1FE5
:10045000CC0FDD1F8D2FBAD68C2FB8D6289ADF91FE
:10046000CF9108956091850180E090E00E94DF0FB8
:100470006091860181E090E00C94DF0FCF93DF93D1
:1004800081E090E00E94C80FC82FD0E0DC2FCC277D
:1004900080E090E00E94C80F9E01282BC901DF91E7
:1004A000CF91CCCF292F332723303105C9F064F405
:1004B0002130310581F02230310509F043C084E557
:1004C00090E024E131E042C021323105F1F02232E6
:1004D000310541F137C082E190E028E631E036C0D5
:1004E00099278130910541F08230910541F0892BA7
:1004F00049F5E0E1F1E005C0ECEEF0E002C0E8EC27
:10050000F0E0849190E09F0121C06330D8F4E62FA1
:10051000F0E0EE0FFF1FE25CFE4F2081318189E0A9
:1005200090E014C0633070F470E0FB01EE0FFF1F29
:10053000E85CFE4F20813181FB01EB5CFE4F808146
:1005400090E004C080E090E020E030E0FA013183E8
:1005500020830895EF92FF920F931F93CF93DF9321
:100560008C0191E0EE24E394F12C461728F1A62F9C
:10057000B0E083E0AA0FBB1F8A95E1F720E030E0EE
:10058000E801C90FD11DF901EA0FFB1FE657FE4F25
:10059000808183304CF08881F701022E01C0EE0F7C
:1005A0000A94EAF7E82BE8832F5F3F4F28303105A4
:1005B00051F76F5F9F5FD9CFDF91CF911F910F915F
:1005C000FF90EF900895DC01EC914E2F50E04D30FC
:1005D000510508F092C0FA01E65CFF4F0C94950FAC
:1005E00011968C9180933201089511962C91119758
:1005F00012968C9190E0982F8827820F911D1ECF24
:1006000011968C91882309F478C0E0913301F09120
:100610003401099411968C91882309F46EC022CF7D
:1006200011968C91882309F468C0EEC313964C91FF
:10063000139712969C9112971196EC918E2F8F73AF
:10064000803108F05AC0983008F057C0E295E6951E
:10065000E695E370E150E33040F4F0E0EE0FFF1F69
:10066000EC5BFE4F2081318102C02DE932E0E82FA2
:10067000F0E083E0EE0FFF1F8A95E1F7E90FF11D2F
:10068000E20FF31F4083089512968C9112971196F2
:10069000EC91E83090F5F0E0E356FC4F808308954C
:1006A00011968C91882349F114C511968C91882359
:1006B00021F12AC513968C91139712969C9112974B
:1006C00011962C9120938801909387018093890142
:1006D0003DC111968C91882381F07BC111968D913B
:1006E0009D91AC9180930A0290930B02A0930C020F
:1006F000089511968C91811170C40895CF93DF9362
:10070000DC0188E0FD0111928A95E9F7E091320160
:10071000EC934E2F50E0FA013197EB30F10508F0E1
:1007200004C1E95BFF4F0C94950F84E011968C9304
:10073000119788E012968C93129790E113969C93F0
:10074000139714968C93149783E015968C93EDC0B1
:1007500046E060E0CD01FEDE83E005C04DE067E0ED
:10076000CD01F8DE84E080933201DFC04FE06EE01F
:10077000CD01F0DE82E0F7CF909185018091860176
:1007800011969C93119712968C93CFC02091820161
:100790003091810190918001822F8295880F880F7E
:1007A000807C432F4295440F407E842B892B1196E9
:1007B0008C931197311120C0C0913001D09131013B
:1007C0001296692F70E053E0660F771F5A95E1F794
:1007D00040E050E0FA01E60FF71FEC0FFD1F8081AB
:1007E0008D934F5F5F4F44305105A1F79F5F90316C
:1007F00001F19093800199C03130C1F7C09130016F
:10080000D09131011296692F70E043E0660F771F97
:100810004A95E1F740E050E0FA01E60FF71FEC0FD0
:10082000FD1F84818D934F5F5F4F44305105A1F7C9
:10083000DDCF10928001311104C081E080938101ED
:1008400074C01092810181E0820F843019F080938E
:10085000820102C01092820180918201813061F098
:1008600040F0823081F0833009F05FC08DE193E089
:1008700005C08DE992E002C085EA93E090933101D2
:100880008093300152C08DE192E0F8CF80917F01DA
:1008900011968C931197E82FF0E0EE0FFF1FEE0FEB
:1008A000FF1FE356FC4F4081518162817381129694
:1008B0004D935D936D937C9315978F5F823019F004
:1008C00080937F0132C010927F012FC0E0E5F1E0FC
:1008D00080E090E022E0280F31910196ED01C80FF1
:1008E000D91F3883332321F08630910599F727E00B
:1008F000A20FB11D1C9219C08091880111968C9392
:1009000011978091870112968C931297809189019B
:1009100013968C930AC020910A0230910B024091E9
:100920000C0211962D933D934C93DF91CF91089536
:10093000249A259A269A279A08952C982D982E98CD
:100940002F9810928401109283010895F6DF809110
:100950008801813009F42F9A0895809184018F3F96
:1009600019F08F5F80938401809188018130B1F408
:100970009091840180918701981302C02E98089568
:1009800080918301882351F020918901921730F0E2
:10099000109284018150809383012E9A0895809152
:1009A00083018F5F80938301089590918801923035
:1009B00079F480FF02C02D9A01C02D9881FF02C0FA
:1009C0002E9A01C02E9882FF02C02C9A08952C986E
:1009D0000895609188018AE092E00E94DF0F6091A3
:1009E00087018BE092E00E94DF0F609189018CE02B
:1009F00092E00C94DF0F8AE092E00E94C80F8330EF
:100A000018F48093880102C0109288018BE092E074
:100A10000E94C80F809387018CE092E00E94C80F6B
:100A200080938901089580E8EAE8F1E0DF011D92F2
:100A30008A95E9F780E1EDE0F2E0DF011D928A9509
:100A4000E9F70895EF92FF920F931F93CF93DF93EF
:100A5000EC0175D38150833048F4E82FF0E0EE0FBD
:100A6000FF1FE65BFE4F2081318102C02DE932E09D
:100A70000DE012E0790180E8E80EF11C60E0762FCD
:100A800040E050E0663008F03FC0F801808190E01F
:100A9000042E02C0959587950A94E2F780FF2DC039
:100AA000F901E40FF51FE081E43038F180E38E0FA7
:100AB000833018F16F5FDE01A70FB11D1296EC9322
:100AC0008E2F90E0FC01E05EF109E830F105A8F41A
:100AD000EE5AFF4F88810C94950F8E5F0DC0805E9B
:100AE0000BC08F5F09C0805F07C08C5F05C0805C52
:100AF00003C0885F01C0805888834F5F5F4F4830D4
:100B0000510511F0762FBECF0F5F1F4F285F3F4F6B
:100B10002E153F0509F0B3CFDF91CF911F910F91B3
:100B2000FF90EF9008952F923F924F925F926F92B5
:100B30007F928F929F92AF92BF92CF92DF92EF926D
:100B4000FF920F931F93CF938C016B01F8D28150CA
:100B5000833048F4E82FF0E0EE0FFF1FE65BFE4F16
:100B60008081918102C08DE992E02DE0E22E22E0A9
:100B7000F22E3C014C0180E8880E911CAA24A3941B
:100B8000B12C212C312CF701808190E0022C02C085
:100B9000959587950A94E2F780FF50C0F301E20D26
:100BA000F31DC081C13E99F060F4C33D38F4C03DEF
:100BB00008F044C0C33008F441C021C0C03E99F0E1
:100BC0001EC0C53E21F078F0C83EC8F40CC0F60146
:100BD000808190E020E22C0F02C0959587952A95A0
:100BE000E2F780FFDCDEC05EC5010C2E01C0880F7D
:100BF0000A94EAF7F8019081892B80831FC04C2E5C
:100C0000469446944694512CC770F601E40DF51DA8
:100C1000818190E00C2E02C0959587950A94E2F7A9
:100C200080FFBDDEF801E40DF51DC5010C2E01C0ED
:100C3000880F0A94EAF79181892B8183FFEF2F1A9D
:100C40003F0A88E02816310409F09DCFEFEFEE1A35
:100C5000FE0AF8E06F0E711C6814790409F091CF58
:100C6000F8018181887F8183838D887F838FCF91F5
:100C70001F910F91FF90EF90DF90CF90BF90AF90BA
:100C80009F908F907F906F905F904F903F902F90AC
:100C90000895FC01808189CEFC01808186CE5F921F
:100CA0006F927F928F929F92AF92BF92CF92DF927C
:100CB000EF92FF920F931F93CF93DF93CDB7DEB7E1
:100CC00028970FB6F894DEBF0FBECDBF80E1EDE0F0
:100CD000F2E0DF011D928A95E9F78F018AE8A82EDC
:100CE00081E0B82E512C98E0792EFE0131967F01DB
:100CF0006624639425E0922ECC24C394D12C48EC36
:100D0000842EE52DE695E695E695F0E0E65FFD4F4D
:100D1000808190E0252D277002C0959587952A95B2
:100D2000E2F780FD52C0852D64D25E9A5E98D701AD
:100D3000E72D1D92EA95E9F7862D8A95F1F74B9BF1
:100D400069824A9B6A82499B6B82489B6C82379B73
:100D50006D82369B6E82359B6F82349B6886B701AD
:100D6000F50120E030E0922FDB018D91BD01882359
:100D700019F08081815002C080818F5F8083AF0134
:100D8000808187FF02C0108203C086300CF0908201
:100D90003196DA018C91833054F0A601092E01C0FE
:100DA000440F0A94EAF7D8018C91482B4C932F5F9B
:100DB0003F4F28303105B9F614D25E9A5E98BFE0F5
:100DC0005B1619F0882D8A95F1F753940F5F1F4F2A
:100DD000E8E0AE0EB11CF0E15F1293CF28960FB69B
:100DE000F894DEBF0FBECDBFDF91CF911F910F9161
:100DF000FF90EF90DF90CF90BF90AF909F908F903B
:100E00007F906F905F900895AF92BF92CF92DF92E4
:100E1000EF92FF920F931F93CF93DF934DE952E030
:100E200020E1B12CD12C80E090E0FA01E80FF91F0D
:100E30003081313021F0323019F4D39401C0B394B1
:100E400001968830910589F72150485F5F4F211145
:100E5000EACFC0E0D0E00FEF13E0E12CF12CC801A5
:100E60008E199F0982309105C0F196958795EC0106
:100E7000CE0DDF1DCE01E2DA8FE891E00197F1F7A8
:100E800000C0000070E2C72E0ADFCA94E9F72AE822
:100E900031E06DE972E040E080E090E0F901E80FB8
:100EA000F91F508153303CF0FB01E80FF91F5081CE
:100EB000543008F04F5F01968830910579F7285F2C
:100EC0003F4F685F7F4F92E02A30390729F74D1571
:100ED00010F07E01C4CF8E01C2CF8E01EE24EA94C1
:100EE00053E0F52EC12CD12C97012C193D0922304D
:100EF0003105C0F1E901D695C795CC0DDD1DCE01B8
:100F00009DDA8FE891E00197F1F700C0000040E220
:100F1000A42EC5DEAA94E9F78AE891E06DE972E0B3
:100F200040E020E030E0FC01E20FF31F508153303D
:100F30003CF0FB01E20FF31F5081513009F44F5F89
:100F40002F5F3F4F2830310571F70896685F7F4F5C
:100F500022E08A30920729F74B1510F06E01C4CFBA
:100F60007E01C2CFCE01801B910B24E09695879520
:100F70002A95E1F76FE070E0C7D7800F911F5EDA26
:100F8000DF91CF911F910F91FF90EF90DF90CF9065
:100F9000BF90AF90DBCC2DE932E04AE851E080E031
:100FA00090E0FA01E80FF91F6081633034F0F90135
:100FB000E80FF91F6081643070F401968830910564
:100FC00081F7285F3F4F485F5F4F83E02D3138073F
:100FD00031F780E0089581E0089543E050E06DE04E
:100FE00072E08AE092E0DCC743E050E06DE072E03E
:100FF0008AE092E0BDD780910A028F3F71F4809120
:101000000B028F3F51F480910C028F3F31F410920C
:101010000A0210920B0210920C020895AF92BF9236
:10102000CF92DF92EF92FF920F931F93CF93DF93B4
:10103000EB015C0120E8A20EB11C6C01F8E0CF0EC0
:10104000D11C7E018C010F5F1F4FA2D78F3F09F487
:1010500080E0F70181937F01C8010C151D0591F710
:1010600028960A151B0549F7DF91CF911F910F9123
:10107000FF90EF90DF90CF90BF90AF900895AF9228
:10108000BF92CF92DF92FF920F931F93CF93DF9384
:101090008C01EB0180E1F82E6E0188E0C80ED11CB6
:1010A000C80169915C012FEFA21AB20A88D7C50165
:1010B000CC15DD05B1F7085F1F4FFA9469F7DF9192
:1010C000CF911F910F91FF90DF90CF90BF90AF9085
:1010D000089548E050E062E072E08DE993E048D77F
:1010E0006DE972E082E090E099DF65EA73E082E802
:1010F00090E094DF6DE172E082E091E08FDF6DE1DE
:1011000073E082E891E08ACF48E050E062E072E06C
:101110008DE993E045D76DE972E082E090E0AFDFC2
:1011200065EA73E082E890E0AADF6DE172E082E0B8
:1011300091E0A5DF6DE173E082E891E0A0CFEDE002
:10114000F2E04DE952E090E0619170E020E030E0A3
:10115000DB01022E02C0B595A7950A94E2F7A0FF25
:101160000FC0DA01A20FB31F8C91813D31F0823D97
:1011700031F0803D29F4916003C0926001C0946019
:101180002F5F3F4F2830310519F7485F5F4F83E0ED
:101190004D315807C9F6992371F0EDE9F3E028E0E5
:1011A0002E0F8191382F32953F70391302C08F7006
:1011B00008952E13F6CF80E00895219A209A229A5E
:1011C00084E58CBD8DB581608DBD08958EBD0DB457
:1011D00007FEFDCF8EB50895549A579A559A569AA0
:1011E00008955F985C9881E15F9A5F988150E1F77C
:1011F00008955F985C985C9A5F9A5F985C9890E01D
:10120000981721F05F9A5F989F5FFACF089584E066
:1012100089BD86E089BD09B400FEFDCF8091D8006C
:101220008F7D8093D8008091E00082608093E00001
:101230008091E00081FDFCCF0895CF92DF92EF9284
:10124000FF920F931F93CF93DF93EC018B017A01F1
:10125000C9D1811133C0E114F10439F0F701808163
:101260009181081B190BC80FD91FC12CD12C011556
:10127000110519F18091E80085FD16C08091E80004
:101280008E778093E8001AD4E114F10449F0F70155
:1012900080819181C80ED91ED182C08285E00EC0A6
:1012A000A1D1882321F30AC089918093F1000150D4
:1012B0001109FFEFCF1ADF0ADACF80E0DF91CF917B
:1012C0001F910F91FF90EF90DF90CF9008952091A4
:1012D0002F04309130042617370748F06115710547
:1012E00039F42091E8002E772093E80001C0B9017D
:1012F00040E06115710581F1209128042223E9F174
:101300002530E9F12091E80023FD35C02091E80067
:1013100022FD2BC02091E80020FFEBCF2091F200AE
:1013200030E0FC01CF016115710559F02032310523
:1013300040F481918093F100615071092F5F3F4F1C
:10134000F1CF41E02032310509F040E02091E80082
:101350002E772093E800CDCF4111CECF06C08091EB
:101360002804882351F0853051F08091E80082FFF5
:10137000F6CF80E0089581E0089582E0089583E04B
:1013800008956115710529F42091E8002B772093C9
:10139000E800FC016115710521F180912804882382
:1013A00041F1853041F18091E80083FD20C08091BA
:1013B000E80082FFEFCF8091F200882331F0809126
:1013C000F100819361507109B1F78091E8008B774A
:1013D0008093E800DFCF80912804882351F0853086
:1013E00051F08091E80080FFF6CF80E0089581E021
:1013F000089582E0089583E0089520912F043091AC
:1014000030042617370748F06115710539F420912B
:10141000E8002E772093E80001C0B901FC0120E02C
:101420006115710569F1809128048823D1F1853017
:10143000D1F18091E80083FD32C08091E80082FD07
:1014400028C08091E80080FFEBCF8091F20090E00F
:101450006115710559F08032910540F42491209373
:10146000F1003196615071090196F2CF21E0809729
:1014700009F020E08091E8008E778093E800D0CFDB
:101480002111D1CF06C080912804882351F08530E6
:1014900051F08091E80082FFF6CF80E0089581E06E
:1014A000089582E0089583E00895982F953058F5C7
:1014B0009093E900981739F07091EC002091ED00BD
:1014C0005091F00003C0242F762F50E021FF19C067
:1014D0003091EB003E7F3093EB003091ED003D7F8B
:1014E0003093ED003091EB0031603093EB0070935E
:1014F000EC002093ED005093F0002091EE0027FFC8
:1015000007C09F5FD3CF8F708093E90081E008957B
:1015100080E00895EF92FF920F931F93CF93DF9394
:10152000E62EEC018C010C5F1F4FF12CFE1499F19B
:101530009881992359F1F801208169817A81319745
:101540003081892F8F70853010F080E025C02230E7
:1015500010F442E001C046E0E8E0F0E020E0E617E9
:10156000F70720F42F5FEE0FFF1FF9CF2295207FA2
:10157000422B232F2295220F220F207C991F99277F
:10158000991F622F692B91DF8823F9F2F394259636
:101590000B5F1F4FCBCF81E0DF91CF911F910F9158
:1015A000FF90EF9008958091290487FF11C08091EA
:1015B000E80082FD05C0809128048111F8CF11C098
:1015C0008091E8008B770BC080912804882349F034
:1015D0008091E80080FFF8CF8091E8008E778093BB
:1015E000E80008952091E4003091E50095E64091EF
:1015F000EC00842F817040FF22C08091E80080FDC4
:101600001CC080912804882391F0853091F080914E
:10161000EB0085FD10C04091E4005091E5004217B9
:10162000530729F39A01915011F784E0089582E05D
:10163000089583E0089581E0089580E00895409141
:10164000E80042FFDECF08953FD041D08091D8001E
:101650008F778093D8008091D80080688093D800DD
:101660008091D8008F7D8093D80084E089BD86E08A
:1016700089BD09B400FEFDCF109228041092250404
:101680001092260442E260E080E00FDF8091E100EA
:101690008E7F8093E1008091E20081608093E20080
:1016A0008091E20088608093E2008091E0008E7F6C
:1016B0008093E0000895E3E6F0E080818E7F8083F0
:1016C00081E080932704C0CF1092E2000895109229
:1016D000E10008951F920F920FB60F9211242F93DD
:1016E0003F934F935F936F937F938F939F93AF93AA
:1016F000BF93EF93FF938091E10082FF0BC0809135
:10170000E20082FF07C08091E1008B7F8093E100BF
:101710000E947C018091E10080FF18C08091E2006E
:1017200080FF14C08091E2008E7F8093E200809160
:10173000E20080618093E2008091D8008062809313
:10174000D80019BC109228040E945D018091E1002C
:1017500084FF2EC08091E20084FF2AC084E089BD0E
:1017600086E089BD09B400FEFDCF8091D8008F7D51
:101770008093D8008091E1008F7E8093E10080917A
:10178000E2008F7E8093E2008091E200816080938E
:10179000E20080912504811106C08091E30087FD5D
:1017A00002C081E001C084E0809328040E945C01B3
:1017B0008091E10083FF22C08091E20083FF1EC080
:1017C0008091E100877F8093E10082E0809328048C
:1017D000109225048091E1008E7F8093E10080913A
:1017E000E2008E7F8093E2008091E200806180932E
:1017F000E20042E260E080E058DE5FD1FF91EF91CD
:10180000BF91AF919F918F917F916F915F914F9118
:101810003F912F910F900FBE0F901F9018951F931F
:10182000CF93DF93CDB7DEB7AA970FB6F894DEBF9C
:101830000FBECDBFE9E2F4E088E08E0F9091F10099
:1018400091938E13FBCF0E9470018091E80083FF7B
:101850001CC18091290490912A04492F50E04A30FC
:10186000510508F012C1FA01E65AFF4F5EC38038F5
:1018700081F0823809F009C180912D048F70809326
:10188000E9008091EB0085FB882780F91092E90040
:1018900007C080912604882311F082E001C080E017
:1018A0009091E800977F9093E8008093F100109268
:1018B000F100C7C0282F2D7F09F0E7C0882319F059
:1018C000823061F0E2C080912B04813009F0DDC0EC
:1018D000933009F080E0809326042DC080912B0482
:1018E000811129C080912D048F7009F4CEC080939E
:1018F000E9009091EB0090FF1EC090912A04933074
:1019000021F48091EB00806214C09091EB00906113
:101910009093EB0021E030E0A90102C0440F551F75
:101920008A95E2F74093EA001092EA008091EB007A
:1019300088608093EB001092E9008091E800877F37
:1019400083C08111A2C010912B041F778091E30006
:101950008078812B8093E3008091E800877F8093DB
:10196000E80021DE8091E80080FFFCCF8091E30059
:1019700080688093E300111102C082E001C083E01F
:101980008093280482C08058823008F07EC0809105
:101990002B0490912C048C3D53E0950771F583E066
:1019A0008A838AE289834FB7F894DE01139620E098
:1019B0003EE051E2E32FF0E050935700E49120FF26
:1019C00003C0E295EF703F5FEF708E2F90E0EA303A
:1019D00010F0C79601C0C0968D939D932F5F243160
:1019E00049F74FBF8091E800877F8093E8006AE263
:1019F00070E0CE0101966BDC13C0AE014F5F5F4F0C
:101A000060912D040E945202BC01009709F43DC070
:101A10009091E800977F9093E80089819A81EDDCAE
:101A20008091E8008B778093E8002FC0803869F5BB
:101A30008091E800877F8093E8008091250480935F
:101A4000F1008091E8008E778093E800ACDD1DC046
:101A500081111BC090912B049230B8F48091E80062
:101A6000877F8093E800909325049DDD8091250475
:101A7000811106C08091E30087FD02C081E001C0B2
:101A800084E0809328040E945E018091E80083FF37
:101A90000AC08091E800877F8093E8008091EB0086
:101AA00080628093EB00AA960FB6F894DEBF0FBE5B
:101AB000CDBFDF91CF911F9108950895CF9380916D
:101AC0002804882399F0C091E900CF709091EC0030
:101AD000892F817090FD80E8C82B1092E9008091D9
:101AE000E80083FD9CDECF70C093E900CF9108959C
:101AF0006F927F928F929F92AF92BF92CF92DF921E
:101B0000EF92FF920F931F93CF93DF9300D01F921A
:101B1000CDB7DEB77C01CDB6DEB68091E80083FF9D
:101B200006C1F701808190E020912D0430912E04B0
:101B30002817390709F0FBC080912A04833009F483
:101B40009DC030F4813071F0823009F4D4C0EFC010
:101B50008A3009F4B8C08B3009F4A1C0893009F08B
:101B6000E6C04EC080912904813A09F0E0C08DB6EC
:101B70009EB61A82198280912B0410912C048B83BB
:101B8000F7018085482F50E08DB79EB7841B950BD9
:101B90000FB6F8949EBF0FBE8DBFEDB7FEB731965E
:101BA0005F0160E070E0CF01DCD14FEF410F8E01AB
:101BB0000F5F1F4F9501BE016D5F7F4FC7010E94F0
:101BC0009E01F70186819781009721F0408550E0C2
:101BD000B501BED11092E9008091E800877F809323
:101BE000E80069817A81C50172DB8091E8008B771A
:101BF0008093E8000FB6F8949EBE0FBE8DBE97C0CE
:101C000080912904813209F092C0ADB6BEB6009130
:101C10002F041091300470902B0460902C048DB729
:101C20009EB7801B910B0FB6F8949EBF0FBE8DBF61
:101C3000EDB7FEB731964F018091E800877F809322
:101C4000E800B801CF019DDB8091E8008E7780939A
:101C5000E80021E0711001C020E030E0021B130B0E
:101C6000280D391D4FEF460D672DC7010E94C00199
:101C70000FB6F894BEBE0FBEADBE59C08091290408
:101C8000813A09F054C08091E800877F8093E80092
:101C90008091E80080FFFCCFF701818540C08091F2
:101CA0002904813209F043C08091E800877F809346
:101CB000E80079DC90912B0481E0911101C080E073
:101CC000F701818734C080912904813281F58091A8
:101CD000E800877F8093E80066DC80912B04909178
:101CE0002C04882736E0969587953A95E1F7F70119
:101CF000958784871CC080912904813AC1F4809122
:101D0000E800877F8093E8008091E80080FFFCCFA7
:101D1000F701848595859695879596958795809307
:101D2000F1008091E8008E778093E8003CDC0FB6EC
:101D3000F894DEBE0FBECDBE0F900F900F90DF91D6
:101D4000CF911F910F91FF90EF90DF90CF90BF90B8
:101D5000AF909F908F907F906F900895FC0139967F
:101D600027E0DF011D922A95E9F721E0FC01218798
:101D700024EF31E03587248723E0248361E0019656
:101D8000C9CB4F925F926F927F928F929F92AF9248
:101D9000BF92CF92DF92EF92FF920F931F93CF9358
:101DA000DF9300D01F92CDB7DEB77C01ADB6BEB6D3
:101DB00080912804843009F08EC08091E4009091D5
:101DC000E500F701228533852817390709F483C018
:101DD00081818F708093E9008091E80085FF7BC04E
:101DE0008DB69EB6408550E08DB79EB7841B950B8F
:101DF0000FB6F8949EBF0FBE8DBFEDB7FEB73196FC
:101E00006F011B821A82198260E070E0CF01A9D0B5
:101E10008E010F5F1F4F960140E0BE016D5F7F4F47
:101E2000C7010E949E01482EF70184859585892B64
:101E300051F091E080E026853785232B09F090E072
:101E4000092F182F02C000E010E0F70166807780AC
:101E50006114710489F049815A81B301C6016BD0C4
:101E600055245394892B09F4512CF701408550E0F7
:101E7000B601C3016DD001C0512C89819A81892B93
:101E8000F1F0411004C0511002C0012BC1F0F70164
:101E9000848595859787868781818F708093E900F7
:101EA0008B8181118093F10069817A8140E050E05B
:101EB000C601C3D98091E8008E778093E8008091B5
:101EC000E4009091E500F701938782870FB6F894BC
:101ED0009EBE0FBE8DBE0FB6F894BEBE0FBEADBE89
:101EE0000F900F900F90DF91CF911F910F91FF9066
:101EF000EF90DF90CF90BF90AF909F908F907F90AA
:101F00006F905F904F9008950024552704C0080EED
:101F1000591F880F991F009729F076956795B8F398
:101F20007105B9F7802D952F0895EE0FFF1F0590CD
:101F3000F491E02D0994FB01DC0104C08D91019026
:101F4000801921F441505040C8F7881B990B08951F
:101F5000FB01DC0102C001900D9241505040D8F7C6
:101F60000895DC0101C06D9341505040E0F70895A1
:101F7000DC01CB01FC01F999FECF06C0F2BDE1BD49
:101F8000F89A319600B40D9241505040B8F7089538
:101F9000F999FECF92BD81BDF89A992780B5089531
:101FA000DC01A40FB51F4150504040F0CB01840F1D
:101FB000951F2E9105D041505040D8F70895262FF7
:101FC000F999FECF92BD81BDF89A019700B402162F
:101FD00039F01FBA20BD0FB6F894FA9AF99A0FBEDD
:061FE0000895F894FFCF04
:101FE60002821900000156011900000000000000DD
:101FF6000183080000016F010800000000000000D6
:1020060000810800000177010800000000000000C0
:102016009D020200182520BE58027A019A01260167
:102026003F015801A5031D021D03A5031D021D0343
:06203600302E362E3700AB
:00000001FF
